:10000000E00501204D3F0000493F0000493F00004E
:10001000493F0000493F0000493F00000000000048
:10002000000000000000000000000000493F000048
:10003000493F000000000000493F0000493F000028
:10004000493F0000493F0000493F0000493F000090
:10005000493F0000493F0000493F0000493F000080
:10006000493F0000493F0000493F0000253600009D
:10007000493F0000493F0000493F0000493F000060
:10008000493F0000493F0000493F0000493F000050
:10009000493F0000493F0000493F0000493F000040
:1000A000493F0000493F0000493F0000493F000030
:1000B000493F0000493F0000493F0000493F000020
:1000C000493F0000493F0000493F0000493F000010
:1000D000493F0000493F0000493F0000493F000000
:1000E000493F0000493F0000000000000000000000
:1000F00000000000D92B0000493F0000493F0000EC
:10010000493F0000493F0000493F0000493F0000CF
:10011000493F0000493F0000493F0000493F0000BF
:10012000493F0000493F0000493F0000493F0000AF
:10013000493F0000493F0000493F0000493F00009F
:10014000493F0000493F0000493F0000493F00008F
:10015000493F0000493F0000493F0000493F00007F
:10016000493F0000493F0000493F0000493F00006F
:10017000493F0000493F000000000000000000006F
:10018000352800003D280000452800004D280000CB
:1001900000000000493F0000493F0000493F0000C7
:1001A000493F0000493F0000493F0000493F00002F
:1001B000493F0000493F0000493F0000493F00001F
:1001C000493F0000493F0000493F0000493F00000F
:1001D000493F0000493F0000493F0000493F0000FF
:1001E000493F0000493F0000493F0000493F0000EF
:1001F000493F0000493F0000493F0000493F0000DF
:10020000493F0000493F0000493F0000493F0000CE
:10021000493F0000493F0000493F0000493F0000BE
:10022000493F0000493F0000493F0000493F0000AE
:10023000493F0000493F0000493F0000493F00009E
:10024000493F0000493F0000493F0000493F00008E
:10025000493F0000493F0000493F0000493F00007E
:10026000493F000010B5054C237833B9044B13B156
:100270000448AFF300800123237010BD78000020F4
:10028000000000007851000008B5034B1BB1034982
:100290000348AFF3008008BD000000007C00002090
:1002A0007851000070B50D461646044610B1081E80
:1002B00018BF01200549064B34229847236832466F
:1002C00029462046BDE87040184700BF144A000088
:1002D0003929000038B50C46054610B1081E18BF74
:1002E00001200749074B4022984701232C602360D7
:1002F000112363604FF4FC43A360002038BD00BFAE
:10030000284A00003929000038B5044600380C4B53
:100310000D4618BF01200B494FF4E072984723683F
:10032000AB4208D04BB9084B25602046984740F2B5
:10033000B273A36138BD0020FCE76FF01100F9E74C
:10034000392900003F4A0000A935000003468068B3
:10035000427B6FF30412427393F927202AB1427B48
:10036000C2F3C00161F3C7124273C2690AB199694D
:100370001047704703468068427B6FF34512427313
:1003800093F927202AB1427BC2F3C00161F3C7125F
:100390004273026A0AB1996910477047F8B50D4671
:1003A000846B114B0646174600210222A868984725
:1003B00021222B7B2270222262700022A380678080
:1003C0000A4BA271E27121463046984750B1084B62
:1003D000304698476B7B03F07B0363F07F036B73BE
:1003E0006FF00500F8BD00BF45320000212D000070
:1003F0004D2D00004A681F4B9A4270B5054637D113
:100400008C68627BD1060ED52069216B8369994285
:1004100026D1238F013B9BB2238723B963F30412B8
:100420006273154B9847627B93060ED56069616BCA
:100430008369994218D1638F013B9BB2638723B9CB
:1004400063F3451262730C4B9847617B11F03001E6
:100450000ED104F124022846084BBDE8704018472D
:10046000236364232387DEE7636364236387ECE706
:1004700070BD00BFF5030000F52700002134000027
:1004800070B5427B8B7B9A420D460BD1037CDB0619
:1004900008D58B695A7802F0FD01202902D1446801
:1004A000214804B970BD6168814201D02468F8E731
:1004B000998894F90C608E4203D094F90E60B14291
:1004C000F4D1202A1BD1194B20469847184B984746
:1004D00095F9273033B1637B03F07B0363F07F032F
:1004E000637305E0134B0122214698470028D9D0B9
:1004F000A369002BD6D02046BDE87040184795F977
:1005000027203AB1637B43F080036373637B6FF30F
:100510008203E5E75B8813F00102637B14BF43F0BD
:10052000080362F3C303F0E7E5050000B1340000FF
:10053000913400009D0300002DE9F0470446006956
:1005400030B1214B9847214B206998470023236104
:10055000606930B11C4B98471C4B60699847002379
:100560006361637B1A4E13F0020FC3F3400104F181
:100570000C0707D130223846B047FF232373A373FB
:10058000BDE8F087DFF85490DFF85480114D204625
:10059000C847C047104A0221A8472046C847C0475D
:1005A00004F124020021A847A56930220021384621
:1005B000B047FF232373A373002DE1D020462B46C1
:1005C000BDE8F047184700BFF5270000CD24000024
:1005D000194100002134000000000020B134000067
:1005E000913400002DE9F04F012987B0054690466F
:1005F00000F09E80022900F09880002940F09D8044
:10060000514CA04782462846A047504B98476B7BE9
:10061000D0F814B0DB07814600F19280D8E90001E0
:100620004B4C0422A047064610B96FF009004CE07D
:10063000437903F0F703022BF7D10078D8F80410C0
:1006400004223044A04704900028EED0437903F000
:10065000F703022BE9D13F4B8278D8F80410984772
:10066000737905900A2B1EBF3346049E0493049BA6
:100670009B79022BD9D1049BDB79012BD5D8344649
:100680002078D8F80410344B20449847044638B3F7
:1006900090F803C00CF00303022BF1D18388827819
:1006A0009AF80D102D4F012003909AF80F00C0F317
:1006B00081000290A079CDE900C05846B84738B90A
:1006C0002846274B98476FF01B0007B0BDE8F08F16
:1006D000856094F90230002BB4BF28616861CFE7D0
:1006E000286908B16B691BB91D4B284698479CE7E0
:1006F0001C49DFF884A0D0471B496869D047059B97
:10070000C8F80030049B194A9B782B73B378AB73FD
:100710006B7B43F001036B73154B0221C5E90A356E
:100720004846144B98470020CFE70D4B9847FAE70F
:10073000437B43F002034373F5E76FF00C00C4E71B
:100740006FF00100C1E700BFB13400009134000038
:10075000D1340000EB3400000F3500009922000076
:10076000390500004D030000750300000000002063
:10077000F5030000993300007D26000038B54B7B5F
:10078000DB070C4610D40A4B9847054650B9094B75
:100790000146302204F10C009847FF232373A37312
:1007A000054B6360284638BD6FF01005FAE700BFBF
:1007B0005533000019410000E50500002DE9F04126
:1007C0000F4D104E104F0020A847044688B90F4B1C
:1007D0009847830711D021460D4B012220469847A8
:1007E0000C4B0D480121984720460C4BBDE8F041C9
:1007F000184721463046B847E5E7BDE8F08100BF1D
:100800009D0A0000594A0000054000004D0F0000FD
:10081000710F0000F50F000094000020451000004B
:10082000024A0348034B111D184700BF080000206F
:100830006C050020850A0000044A1168034609B9C6
:10084000034911601068034413607047940200204C
:10085000E0050120891A70B5CC1D48BF01F10E04D6
:1008600000EBE40002F0070210F8011CD418082C79
:1008700041FA02F118DD10F8025CC2F10806B54039
:10088000102C41EA05010FDD10F8030CC2F1100530
:10089000182CC8BFC2F1180200FA05F541EA05019B
:1008A000C4BF00FA02F211434FF0FF30984021EA32
:1008B000000070BD37B50E4B054601A898470D4A9C
:1008C0006B09D90102EBC31351581A6A1C690A4B10
:1008D00054400C4001A8544005F01F0598470120E2
:1008E00000FA05F5254208BF002003B030BD00BF67
:1008F000FD3E0000008000410B3F000013B507489B
:10090000074C0268917F537B003918BF0121009189
:10091000017912688068A04702B010BD98020020DB
:100920007115000038B5002843D1234CE368002B33
:1009300038D0B3F90000421C34D0204BC0B29847E5
:10094000E3685B88984203D00423A376022038BD75
:10095000A07E042801D10123F7E701281FD102233B
:10096000A376174B236101236377002384F82E308D
:100970002379E3B1208EB0FA80F04009114A124980
:10098000124D40F22C53A84700232371104B2360D3
:10099000104B9847A07E831E58425841D7E7032842
:1009A000E6D1D4E7A37E033B012BE1D8D7E70120B2
:1009B000E4E70420CBE700BF98020020B508000060
:1009C000801A0600624A0000754A00009940000043
:1009D000A8020020FD0800002DE9F0410B4D0C4E4F
:1009E0000C4FDFF834803368B0681A8941F20D117A
:1009F0001204B847044628B1B068C047C30502D402
:100A0000013DF0D100242046BDE8F081410D0300F6
:100A100098020020E51300003D15000073B50E4C50
:100A20000E492368A0681A890D4E01251023CDE9CF
:100A300000559A40B04760B12168A068094B2A462A
:100A40000E31984728B1A068074B02B0BDE870404E
:100A50001847002002B070BD98020020091108005C
:100A600009120000F913000099140000034B1979D2
:100A700011B99868024B1847704700BF98020020D0
:100A80008915000010B5044B04249C76FF241C71CA
:100A9000C3E902015A6310BD980200202DE9F04F0E
:100AA0008F4B87B098470128804605D08D4B9847DB
:100AB000404607B0BDE8F08F8B4C8C4F23688C4EBE
:100AC000D87200251D731D818A48B847A0688A4BDB
:100AD0009847A0682A464FF48851B047002839D07B
:100AE000A0684FF4D57245F20851B047002837D1BD
:100AF00000252368DB7AD80740F1FF81DFF810A2D8
:100B0000AD0741F6EF39A068002241F23711B04736
:100B1000002831D179497A48B8477A48B8472368DC
:100B2000A0680222DA724FF488510022B04788B1DF
:100B3000DFF8DC9141F6EE35A068002241F20111A8
:100B4000B047002840F0B780C5F5DF526E496F48C6
:100B50000E32B84723684FF0030883F80A80A5E7F0
:100B6000A0686B4B9847451CC2D0C0F30B00B0F592
:100B7000D57FEFD14546BCE7A0682A4641F229114E
:100B8000B04710B95D496348C6E7A068D04710F088
:100B9000010207D0B9F10109B5D1024657495E48B3
:100BA000B847BAE7A06840F23A51B04710B9534984
:100BB0005A48B1E7A068D047410004D52268D37AEB
:100BC00043F00803D372A068002241F23B11B04702
:100BD0000028BFD02368DB7ADA0740F18E81504BC2
:100BE00098470028B6D0D4F800A04E4D0AF10E0B5D
:100BF0000823602280215846A847404BC0F3C30217
:100C000000F0070003EB800003EB82028021D36F2A
:100C1000026E53434FF47A725343CAF800307E2277
:100C200002235846A847A946002800F04C81162305
:100C3000302280215846A84701304002BAF80820E7
:100C4000CAF804001204A06841F23711B047002826
:100C500080D00125CDE900553349A068DFF8D8A040
:100C600008230022D04700283FF474AFA0682F4B20
:100C70002A4604A9984700283FF46CAFA0682C4B83
:100C8000984700283FF466AF04233822402104A887
:100C9000C847A842D4F800A000F02C81022840F0F8
:100CA00037812B462F22402104A8C84701280CBFBA
:100CB000302320231FE1A068C84710F0010206D0AE
:100CC000013DBFF439AF10491A48B84742E7A06860
:100CD00040F23A51B04788BB0B491048F5E700BFD6
:100CE000250900006D0A0000980200200540000060
:100CF000E5130000794A0000491500005C4B000034
:100D0000914A0000F24A00006B4B0000064B0000C5
:100D10003D150000A24A0000B44A0000E14A00006C
:100D20001D0A00005508000033110800F9130000E7
:100D3000991400002A4B000009120000A068C8475F
:100D400000F0C040B0F1804F08BF2268A06802BF29
:100D5000D37A43F00803D37241F23B110022B0472B
:100D600000283FF4F7AE704B984700283FF4F2AEEE
:100D7000D4F800906D4D09F10E0B04237A228021E6
:100D80005846A8470138AA46032803D8DFE800F0F0
:100D900091939597122389F80C30602208238021C3
:100DA0005846D047624BC0F3C30200F0070003EB84
:100DB000800003EB82028021136A026E53434FF4DA
:100DC0007A725343C9F800303E220C235846D0476C
:100DD00040F6FF739842054612D003232F2280214C
:100DE0005846D0476B1C023003FA00F5502204230A
:100DF00080215846D04705FA00F0800AC9F804005F
:100E000099F80C303F2B3ED901230022CDE9003266
:100E10004849A068484D4FF40073A84700283FF4A4
:100E200099AEDFF824B13225D946A06803A9D84786
:100E300000283FF48FAE013DADB2002DF5D1206802
:100E40000C233E2280210E30D04740F6FF7398429B
:100E500037D10425A06804A9C84700283FF47AAE1A
:100E6000013DADB2002DF5D1049B22685B085360B3
:100E70003625A06804A9C84700283FF46BAE0135A9
:100E8000ADB2802DF5D1A0684FF4007241F210117F
:100E9000B04700283FF45EAE284B984700283FF447
:100EA00059AE274B98472748B847236800229A72C3
:100EB000FCE514236FE722236DE730236BE7402323
:100EC00069E73225D5E70C233E2280215846A84702
:100ED000032305462F2280215846C847013502309A
:100EE00085400423502280215846C84705FA00F067
:100EF000800AA3E61A238AF80C302368DB7A03F011
:100F00000903012B06D02368DB7ADB07C4D4C8E7CA
:100F10001023F0E7A0684FF4007241F21011B047BF
:100F20000028F0D116E600BF1D0A00005508000099
:100F30005C4B00000811080009120000D9090000EC
:100F4000FD080000454B00009D14000008B5054B4E
:100F5000984728B9044B9847044B1B68D87A08BDBA
:100F60000020FCE7250900006D0A0000980200201F
:100F7000F7B5174B0F4614469847054628B9154B49
:100F8000984728B9144B98470525284603B0F0BD6B
:100F9000124B134E1349B068012C98BF19463368A1
:100FA000DB7A1B0758BF7F020123CDE900433A4695
:100FB0004FF400730C4FB8470028E3D00B4BB068D8
:100FC00098470B4B0340002BDCD134863487DCE799
:100FD00025090000D90900006D0A00001111080060
:100FE0009802002012111000091200003D150000A7
:100FF000000058E4F8B50E4D0E4A0F4F0646288EF5
:101000000C46A04234BF002001200C494FF4D963A4
:10101000B847A8680A4B22463146984728B1288E1F
:10102000011B89B200202986F8BD01460520FAE798
:1010300098020020624A000099400000754A0000B2
:10104000F913000038B5124D124B0446A8689847B2
:10105000E0B144B100232B862B8F012B08D10E4B1E
:101060009847002038BD2B8E002BF5D02046F9E79D
:101070000022A868094C43F20C11A0470246002840
:10108000EDD1A86843F20C11A047E8E70520E9E795
:1010900098020020991400006D0A0000E51300007A
:1010A000F7B5FF230546174E8DF8063001220DF1E6
:1010B00007018DF80730144F144CB04701220DF191
:1010C00006012846B84701220DF107012846B0471E
:1010D00001220DF106012846B84701220DF1070152
:1010E0002846B04701220DF106012846B847013CC9
:1010F00006D09DF80630FF2BEFD1012003B0F0BDE4
:101100002046FBE7C1160000CD160000410D03008C
:1011100013B5FF2304468DF803300DF10301054B91
:1011200001229847044B022201A92046984702B0A9
:1011300010BD00BFC1160000CD1600002DE9F74517
:10114000254A2649264D274C274FDFF8B8A0FF2314
:101150008DF80730064693881068B0FBF3F203FB66
:101160001200B0FA80F0A823204A4009A8470023C3
:101170008DF80630013C05D11D491E481E4B98478D
:1011800020461FE001220DF107013046B847012239
:101190000DF106013046D0479DF8060010F0F0082A
:1011A00015D1003818BF01200C49104ABE23A847AA
:1011B0009DF806000E49104B10F0070405D00F48AB
:1011C0009847404603B0BDE8F0850D48D7E7FE28B4
:1011D000D0D10120F6E700BFD4020020754A0000FC
:1011E0009940000021A10700C1160000184C000022
:1011F0006F4E00002F4C000005400000494C0000DD
:10120000644C0000CD1600002DE9F04F89B00F4668
:101210000293FF231646644C644A8DF815308DF80E
:1012200017306349E823054607F03F0AC7F300205B
:10123000A0474AF040038DF81830330E8DF819306E
:10124000330C8DF81A300DF1180C330A8DF81B3061
:101250008DF81C60062200236446013A12F0FF025A
:1012600030D15B0043F00103DFF86C918DF81D3045
:1012700001220DF115012846C847214606222846BD
:10128000C847DFF85881FF2301220DF116012846D7
:101290008DF81630C047072401220DF116012846AB
:1012A000C0479DF916309DF81620002B1EDA013C30
:1012B00014F0FF04F0D13F493F48334652463F4DBA
:1012C000A84723E01CF8010B08215B00DBB283EA8E
:1012D000000E1EF0800F01F1FF3118BF83F00903EB
:1012E000400011F0FF01C0B2EFD1B6E7DFF8F0B077
:1012F00012F00803CBF8082003930BD02D49304897
:101300000092334652462D4CA0470024204609B097
:10131000BDE8F08F12F0040405D000922549294859
:1013200033465246EFE712F0FE0F07D000922149F4
:10133000224D254833465246A847E7E7B90409D568
:10134000224A28469047044620B91A492048334685
:101350005246B4E7BA050BD50022CBF808200DF1B0
:10136000170101222846C8471A4901222846C047CA
:101370007B050DD501220DF117012846C84704222F
:1013800014492846C047DBF8082012BACBF80820D9
:10139000BDF84820029BABF806200022ABF80430D1
:1013A000CBF800200124B1E799400000184C000060
:1013B000314D0000C84E0000544D000005400000B3
:1013C0007C4D0000B34D0000EC4D0000A11000006A
:1013D0001B4E0000DC020020C1160000CD160000EC
:1013E000D402002013B50023CDE90033014CA047FF
:1013F00002B010BD091200002DE9F74FFF231E4D6A
:10140000DFF88890DFF888A08DF807300646884618
:10141000144600271CB9012003B0BDE8F08FB5F8D1
:1014200006C02B68A888B3FBF0F0844594BF002069
:10143000012040F253134A465146DFF858B0D847CE
:101440000E4B30469847013CA4B20028E4D00DF181
:1014500007010B4B012230469847AA88094B08EB3D
:10146000070130469847AA882B6813442B60304602
:10147000054B17449847CDE7D40200203D110000EA
:10148000C1160000CD16000011110000184C00001C
:10149000754A000099400000012070477FB51F4C3D
:1014A0001F4AE6880191FF238DF80F300546236817
:1014B000A088B3FBF0F086421A491B4E40F2B713E6
:1014C00094BF00200120B047A2882368B3FBF2F14B
:1014D00002FB1133B3B1154B01220DF10F01284668
:1014E000984704220DEB0201114B284698472368C8
:1014F000A28804332360B3FBF2F102FB113343B142
:10150000012004E00B4B284698470028E3D104B0A3
:1015100070BD094B28469847F2E700BFD40200206F
:10152000184C0000754A000099400000C1160000E8
:10153000CD1600003D11000011110000014B98680C
:10154000704700BFD402002073B5FF23074E8DF80B
:10155000073005460A2401220DF107012846013C07
:10156000B04714F0FF04F6D102B070BDC116000000
:10157000044AD2F8903023F08053C2F89030002013
:10158000704700BF00800041044AD2F8903043F019
:101590008053C2F890300020704700BF00800041A7
:1015A00038B50D46044610B1081E18BF01200A497F
:1015B0000A4B402298472046094B40F8045F2946D1
:1015C0009847002807DB4FF40043A382054B2361B3
:1015D000054BE360002038BD364F0000392900007C
:1015E000D93C0000891600005116000010B50446D1
:1015F0000038054B054918BF012057229847201D88
:10160000034BBDE81040184739290000364F000051
:101610000D3E000030B50C4685B0054610B1081EE1
:1016200018BF0120B3220749074B9847236801934D
:1016300063680293A368039301A9044B281D98478C
:1016400005B030BD364F0000392900003D3E000096
:101650007FB50446003818BF01200E4615460749DD
:10166000074BA32298470023CDE9016301A9054B4D
:101670000395A4F10C00984704B070BD364F0000EC
:1016800039290000151600007FB50446003818BF40
:1016900001200E4615460749074B8722984700232D
:1016A000019301A9054B0296A4F10C0003959847FC
:1016B00004B070BD364F0000392900001516000037
:1016C000014B0C30184700BF51160000014B0C3085
:1016D000184700BF8916000070B5084C0849094E2C
:1016E000251D602304F180022846B04704F144011F
:1016F0002846054BBDE87040184700BFE0020020B7
:10170000A8050020C53200007D07000070B50D4619
:10171000044610B1081E18BF01200549054B3122AF
:10172000984729462046044BBDE87040184700BF43
:10173000524F000039290000092A000083780B422B
:10174000FCD1704700207047064A002332F8021B84
:10175000814201D358B270470133082BF6D10720DC
:10176000704700BF824F0000426892F88930013311
:1017700082F88930036804221A83704738B50368F9
:101780005D680446D5F88000A04216D895F88A30E6
:1017900003EB830300EBC30084428CBF00200120D5
:1017A0000749084B40F2C2329847D5F88000201A0A
:1017B000054CC010604340B238BD0020F0E700BFC8
:1017C0006C4F000039290000CDCCCCCC90F9893089
:1017D00013B1013B80F8893070470000F8B5046808
:1017E000144B67680E46154698472468C3B204EB4D
:1017F00043105901032280F8072107EB431380F8B7
:1018000009217E505A6865F30D025A605A686FF3D9
:101810009B325A6090F8003103F0FC0343F002035E
:1018200080F80031402380F80531102380F804311E
:10183000F8BD00BF7D170000F8B504681F4B656850
:10184000064698472268C3B202EB4311032481F88D
:10185000074181F80941747C580105EB4313CCB969
:10186000174A2A505A6864F30D025A60B0895A68C0
:1018700060F39B325A6091F8003103F0FC0343F0AF
:10188000010381F80031402381F80431102381F8ED
:101890000431F8BDD6E90527F4693C442C5058685A
:1018A0006FF30D00D21B58605868B2F5804F28BF07
:1018B0004FF4804262F39B305860DCE77D170000F4
:1018C000C00300202DE9F0414F4F07F1CC03C7F8CA
:1018D000C03004230C4687F8CA30054610B1081EF4
:1018E00018BF0120494B4A494A4E40F2BE22984750
:1018F000A37813F0010F11D103212046B0472378BC
:101900009B0706D5237803F0FD032370B04702211F
:10191000B0470123237003212046B0470121204610
:10192000B04700223C4BDFF8FC80284698473B49F3
:10193000D7F8C030C5E90411C5E90048002297F87E
:10194000CA00043396465FFA82FC844503F12803FB
:101950004ED34FF40003D3F88420C2F34413C2F3F0
:10196000822112F01F0249D01F2A08BF0922002B32
:1019700046D01F2B08BF1923002943D0072908BFD1
:10198000062143EA821343EA01334FF082429BB2BD
:101990001385D37843F00303D370D37843F00C035B
:1019A000D3701F4BC7F86C5100224FF48031C7F839
:1019B000C420A7F8C82099604FF4003199604FF413
:1019C000802199604FF40021996084232370204680
:1019D0000321B0474FF48063C4F8248023814FF47F
:1019E000047323834FF6EF53A3821046BDE8F081C2
:1019F00043F8281C03F806EC0132A4E70922B6E7F5
:101A00001923B9E70621BCE7C003002039290000EB
:101A10006C4F00003D170000613A000045170000C0
:101A200000E100E000040020F7B50D46174604462B
:101A300028B1406818B12068003818BF0120144E42
:101A40001449154B40F223329847002F18BF3E46E9
:101A50002DB1012D17D06FF00C0003B0F0BD23693C
:101A6000B34212D00D4B01A8984726613FB10C4BF1
:101A7000204698470B4B01A898470020EDE7606887
:101A8000094B9847F6E76661F7E72846E5E700BFA8
:101A9000451700006C4F000039290000FD3E000092
:101AA000691700000B3F0000CD170000F8B5044691
:101AB00000381649164B40F24B3218BF01209847A8
:101AC000616891F988301BB1FF2381F88630F8BD39
:101AD0002568A1F884300126102705EB431090F803
:101AE0000621D20609D4B1F884C006FA03F242EA0C
:101AF0000C02A1F8842080F805710133042BECD18D
:101B0000044B204698470323DFE700BF6C4F0000DB
:101B1000392900006917000090F82630033B072B95
:101B200070B5044621D803685D68437C43B995F9D4
:101B3000883013B1013B85F888300C4B2846984714
:101B4000022384F82630636884F827100BB12046FE
:101B5000984795F9883043B995F98630002B04DA17
:101B60002068034BBDE87040184770BDCD170000DA
:101B7000AD1A000073B50668124B756801910446F2
:101B8000984733680199C0B200F1080203EB421292
:101B90001026567194F90F20002A4FEA401006DBF8
:101BA0000544A2696D68C5F38D352A44A2611844C5
:101BB000032380F80831044B204602B0BDE8704092
:101BC000184700BF7D170000191B00002DE9F74FD3
:101BD000B04DD5F86C4123681A8C92B2002A00F0FF
:101BE0008D81D2B2B2FA82F2C2F11F02511C5FFAA9
:101BF00082FE00F0E18003EB4E1C67689CF8071141
:101C0000D7F880609CF809E102EB8204C8B211F0B9
:101C100020014FEAC4085FFA8EFE06EBC4040AD026
:101C200020238CF807316FF018019B4B204603B03E
:101C3000BDE8F04F184710F0080913D0082307EB50
:101C400042128CF80731D389D18103F00F03082B9E
:101C500014BF6FF005036FF0070384F827306FF0AF
:101C60000501E2E710F0040114D0042307EB42124F
:101C70008CF80731937A03F0FF01002B00F09C8071
:101C800082F80A90637C012B02D0022900F0948034
:101C9000FA23E2E700EA0E00870700F0078103233A
:101CA0008CF807319CF800317C4F019103F003035D
:101CB000012B204640F09280B84794F826300199D5
:101CC000092B02D1764B2046B1E7052B74D156F88B
:101CD0000830B4F80CA0D3F804E0C0B20EEB401307
:101CE0004FEA401B5A68C2F30D029146002A72D097
:101CF000637C002B63D0D4E905C1E3695EF80BE097
:101D0000ACEB010C62450B4428BF624611442CBF6A
:101D10004FF0010C4FF0000C1A44AEEB030E9A4248
:101D200003EB0E0B50D1637C002B52D0A161637C7E
:101D3000002B40F06C824FF4FA736384BCF1000F07
:101D400000F06D8256F808900A2384F8263032237A
:101D50006384D9F80030D9F80460083003EB4013ED
:101D60004FF0010883F805802046B847D9F80020D5
:101D7000C3B202EB43105C01032180F8071106EBAC
:101D8000431380F8091180F8058135515A686FF3C3
:101D90000D025A605A686FF39B325A6090F8003116
:101DA00003F0FC0343F0020380F80031402380F885
:101DB0000531102380F8043103B0BDE8F08F63696A
:101DC000B4F81CC0E18B99E79BF800B003F801BBA5
:101DD000A5E7E183ABE74FF0000CA8E7B84794F81C
:101DE000263001990A2B3FF46DAF062BE4D156F84B
:101DF0000880657CD8F8043015B94FF4FA72628413
:101E0000C0B203EB4010A38940686669C0F30D00BF
:101E1000834282BFE37C6FF38613E3747DB1324665
:101E2000D4E9063658B3034465B1A361934229D37C
:101E3000E17C11F0400125D1002DBDD042E7A28BFD
:101E4000E38BEFE7E383E08BA18B8842EED3E17C69
:101E5000490617D4092384F82630322363842046A8
:101E6000B847D8F80030C0B2083003EB4010012367
:101E700043710C4B204603B0BDE8F04F1847002DCE
:101E8000D4D1E0E7D21AF118074B204603B0BDE8E1
:101E9000F04F1847C0030020751B00007D1700009D
:101EA000191B000039180000DD17000010F01000A9
:101EB0001CD0102201238CF807218CF808218CF803
:101EC0000531A36993F90020002A03DA052384F879
:101ED0002630CEE79A790AB9DB792BB10623A28B9B
:101EE000616984F82630CFE70923F0E7AF49B04BAA
:101EF00040F21B2203B0BDE8F04F18479E8BB5B2ED
:101F000016F0040600F0B380042265689A831B8AE9
:101F100013F0070353D095F98730002B04DD95F9B2
:101F20008630002B3FF748AF2369204603B0BDE859
:101F3000F04F1847D5F8802007FB062292F913309E
:101F4000002B0BDA6068C047D37C6FF3C713D374E0
:101F50002368083603EB461686F80490013195F89D
:101F60008A30CEB2B342E5D895F9863095F987200C
:101F7000002B2BDD013A52B285F88720002A7FF42E
:101F80001BAF60688B4B9847B5F884101346102040
:101F900041FA03F2D50742BF226803F1080502EBBC
:101FA000451203F1010348BF5071042BF0D163695E
:101FB00002220121204603B0BDE8F04F1847DFF8A8
:101FC000F481194628274FF01009C8E7002A1DDDC3
:101FD000013AD2B285F88720002A7FF4EDAE60681E
:101FE000744B9847B5F884101346102041FA03F259
:101FF000D20742BF226803F1080502EB451203F144
:10200000010348BF1071042BF0D1D0E76A4F0026BE
:10201000D5F88000304490F82630032B18D9437C43
:10202000B3B9B0F92230002BC4BF03F1FF334384AE
:10203000B0F92030002BC4BF03F1FF330384B0F9A3
:10204000223013B1B0F9203013B96FF00701B8474F
:102050002836A02EDCD123692046984795F989308F
:10206000002B3FF7A9AE236804229A82A4E615F458
:102070005E7F3FF4A1AE198BD4F8049015F00800F0
:1020800089B266D008229A8399F88A30F7B2BB42A7
:1020900002D8636904228CE7D9F88050282303FB17
:1020A000075595F82630002B4FD095F811A0EA7C03
:1020B00095F80EC0E97BA88995F810B00AF10103E4
:1020C00002F00302012A4FEAC30303F038030CBFF6
:1020D0004FF000084FF0040843EA0803BAF1000F7C
:1020E00035D011F0800F14BF4FF001084FF00208F7
:1020F00043EA080863687A0103EB47170192B7F8CF
:102100000CE02E4B6CF3060EA7F80CE0B7F80CC0F1
:1021100061F30B2CA7F80CC098477B6860F31E7323
:102120007B602368019A1A445FFA88F882F800817C
:1021300082F803B1BAF1000F02D1032385F82630EB
:102140001F4B6FF006012846984701369CE7D046A2
:10215000CEE705EA010616F4007214D04FF440727F
:102160009A834FF41C729A82198921F40071090430
:102170004FF4B872090C19819A831A83A9F8860062
:102180006369024615E7F7051CD54FF48071998203
:102190004FF4007199831983198989B241F48071D0
:1021A0001981A9F88620636903E700BF6C4F00001E
:1021B00039290000CD170000751B000049170000E9
:1021C000191B0000E80608D5CA0506D510229A8317
:1021D0000122154B11462046984716F0700F2368D0
:1021E00013D070229A839A824FF402721A831A894A
:1021F00092B242F480721A81322389F887300B4BF5
:10220000204603B0BDE8F04F18479D83D4E5BCF1EC
:10221000000F02D1CA457FF62CAE002152E5CA4517
:102220003FF690AD25E600BF613A00006917000057
:10223000026813899BB243F400731381704710B591
:1022400004682189237BA48B89B2DBB2A4B2092A5A
:102250001ED8DFE802F005050D1D161D1D1D051910
:1022600004F44070B0F5807F14BF0020012007E027
:10227000436893F986306BB981F48070C0F3002015
:1022800010BDC1F34020FBE703F00C000828EBE78A
:102290000020F5E70120F3E72DE9F04F87B0C3F305
:1022A000C126C3F3090301939DF840A0009107469E
:1022B00001361846814B9DF844909DF848509DF892
:1022C0004CB0904698477D4B0393012E0AF00304CF
:1022D00007D01AF0010200F0D880042E08D10022A5
:1022E000D3E0BBF1000F03D1631E012B98BF022680
:1022F0007B680293724B33F810A0724B05A8984785
:10230000786890F88A1000224FF0280ED3B29942D4
:1023100013D9D0F880300EFB023B9BF826C0BCF1ED
:10232000000F24D09BF80EC0009B9C451FD19BF84A
:102330000F3043451BD1130615D500234FF0280C51
:10234000DAB291420FD9D0F880200CFB032B03F1B5
:10235000010E9BF826B0BBF1000F0AD14FFA83FBA8
:10236000BBF1000F07DA584B05A89847B7E70132D1
:10237000CCE77346E4E70CD1B8F1000F06D0012397
:10238000994240F086804FF0FF3B02E0019B402BDA
:10239000E9D8029AD2F880100BEB8B0301EBC30251
:1023A00041F83370012382F8263005A8464B01928C
:1023B0009847DDE900329373AB00D17C82F80F803F
:1023C00003F00C03334303F01F0321F01F010B4301
:1023D000022DA2F80CA05474D37464D1012C62D1E4
:1023E000B9F1100F28BF4FF0100909F1FF3905FAB4
:1023F00009F5ADB2FF2D28BFFF251574538A157C52
:1024000023F4814323F07F03012E538208BF002170
:1024100004F1010318BF04215FFA8BFB41EAC303F7
:1024200024B118F0800F14BF012402241C437B68E0
:10243000019203EB4B19009AB9F80C1062F30601F4
:10244000A9F80C10B9F80C1068F30B21A9F80C10BE
:10245000039B50469847D9F8043060F31E73C9F8BF
:1024600004303B68019A03EB4B1B0021E4B28BF86C
:10247000004102238BF8035182F827102C218BF89E
:1024800008118BF8091182F82630104607B0BDE814
:10249000F08F92F84E00283210B10133DBB26FE7B3
:1024A0004FFA83FB75E7022C05D1B9F1000F02D179
:1024B00001231374A2E782F810909FE749170000E8
:1024C000824F0000FD3E00000B3F000037B505467F
:1024D00038B10368ABB1186818B15868003818BF34
:1024E00001201649164B40F27A429847154B01A835
:1024F000984795F82640144B2CB901A898472046D8
:1025000007E01846EDE7022C05D001A898476FF0C8
:10251000030003B030BD012285F8262001A89847AA
:102520000A4B284698472B68C0B208301B68400108
:1025300000241C5485F82640E1E700BF6C4F0000E2
:1025400039290000FD3E00000B3F00007D17000010
:102550002DE9F04F884687B091461F4602F00F0BD9
:10256000044638B10368DBB1186818B15868003800
:1025700018BF01203B493C4B40F29C4298472368DE
:1025800005A8D3F804A0394B984794F82660384B37
:1025900046B905A898476FF0130007B0BDE8F08F63
:1025A0001846E7E7022E04D005A898476FF003000D
:1025B000F3E7012284F8262005A898472D4B2046F2
:1025C00098472168C3B203F108000A684001402F10
:1025D000105CC0B204D984F826606FF00C00DCE710
:1025E00000F03800082804D084F826606FF01A0044
:1025F000D3E7214D01913846CDE90223A847DAF807
:1026000004500199039B000725F0E04500F0E040ED
:102610002843CAF80400BAF80C50E07C25F4706531
:102620002D042D0C45EA0B25AAF80C509DF84050BE
:1026300084F80E8065F38300E07484F80F90496895
:10264000A78101EB4311888968F306008881029A0B
:1026500002EB43132C2283F80921002084F8266022
:102660009BE700BF6C4F000039290000FD3E0000D1
:102670000B3F00007D1700004917000038B50446E5
:1026800000380D4618BF01200349044B40F2CF42E9
:1026900098476560002038BD6C4F00003929000064
:1026A0002DE9F3474C4E0446894690461F46B047F5
:1026B00082463CB3206828B105682DB340680038D5
:1026C00018BF0120454D464940F2D352A8475FFA52
:1026D0008AF00328424940F2D4528CBF00200120E6
:1026E000A847657C002D73D13E4B01A8984794F80C
:1026F00026303D4953B901A888476FF0130002B056
:10270000BDE8F0872046DDE72846DBE7022B04D052
:1027100001A888476FF00300F1E70323206884F8DD
:102720002630324B984723685A6892F88830013334
:1027300082F8883001A88847BDF928302384002F0B
:10274000E58314BF4FF4FA734FF0FF3384F827503A
:102750002568A7836384C4E9058920466F68B0476C
:102760002A68A369C0B200F1080102EB41121021EE
:10277000D1711F4A03F10806144613F801CB82F801
:1027800000C0B34202F10102F7D1410107EB401250
:102790007C505368082464F30D03536053686FF34F
:1027A0009B3353602B6803EB401090F8002102F03C
:1027B000FC0280F80021012280F80421402280F8E8
:1027C0000521102280F8042180F80921002096E7D5
:1027D0006FF01A0093E700BF7D1700003929000051
:1027E0006C4F0000FD3E00000B3F00006917000029
:1027F000C003002010B5044638B1006828B1036852
:102800007BB14068003818BF01200749074B40F2F0
:10281000576298472046064BBDE810406FF0020112
:1028200018471846F1E700BF6C4F00003929000037
:10283000751B0000004B1847CD1B0000004B1847CC
:10284000CD1B0000004B1847CD1B0000004B184764
:10285000CD1B00000B4A13889BB243F4807310B564
:102860001380094B094C9847094B9847094B9847E7
:102870000820A047084B9847234640F6F770BDE86C
:102880001040184700400041813500009D2800009D
:102890003F290000CD2B000041290000C20707D5C9
:1028A000094B0A4A1A6243F6FD7259681142FCD17B
:1028B000030707D5044B064ADA6243F6FD725968EE
:1028C0001142FCD1704700BF001C0040060101000E
:1028D00005010100006800B970478842FAD1012063
:1028E0007047000038B5074B0446984780F0010058
:1028F0000D46054B05493922C0B2984723682B6025
:10290000256038BDD528000039290000924F00000D
:1029100071B103688B4204D11B68036001207047CA
:1029200013463BB11A688A42FAD10A681A60F5E781
:10293000084670471846704700B900BE7047704798
:102940002E4B1A6A22F00F0242F004021A6243F67A
:10295000FD7259681142FCD15A68C2F380015207D6
:10296000FAD4274A11774321C3F88010254B93628C
:1029700092F82C30C3F30011DB06F9D4204B82F817
:10298000201093F82C205007FBD402221A771C4BFE
:1029900093F82C209107FBD45A6A5A62184B93F88B
:1029A0002C201207FBD4112283F82020144B93F81B
:1029B0002C205007FBD493F82020D10719D51A6991
:1029C00002F41062B2F5106FF9D10C4A5368002B73
:1029D000FCD1136A23F00F0343F00603136243F69E
:1029E000FD7351681942FCD1044A53685B07FCD45B
:1029F00070471A69D205FCD5E7E700BF001C00400C
:102A000000100040B805010438B50C46054610B169
:102A1000081E18BF0120124B1249D822984794F87B
:102A20002F302C6043F0010384F82F3094F82F00EE
:102A300010F00100FAD10E2384F82E300F2384F811
:102A40002930A38E9BB26FEA53236FEA4323A386F8
:102A5000E38E9BB26FEA93236FEA8323E38638BD4C
:102A600039290000B04F00002DE9F8430E46154605
:102A7000044618B129B3101E18BF01201249134B88
:102A8000134FF12298470834B9462046B84700282A
:102A9000FBD0DFF844800027F15D2046C047204688
:102AA000C8470028FBD00137BD42F5D8002D094E9C
:102AB00008BF01252046B0470028FBD02846BDE8C6
:102AC000F8830846DAE700BFC74F00003929000045
:102AD000BB3C0000C53C0000AD3C00002DE9F843C4
:102AE0000E461546044618B1E9B1101E18BF012064
:102AF0000E490F4BDFF83C90DFF83C804FF48672B4
:102B00009847002708342046C8470028FBD02046B5
:102B1000C047F0550137BD42F5D8002D14BF2846F7
:102B20000120BDE8F8830846E2E700BFC74F000078
:102B300039290000CF3C0000B33C000038B50D46F9
:102B4000044610B1081E18BF01200749074B342264
:102B50009847074B294604F10800984718B9054BD8
:102B60006360054B236038BDC74F00003929000062
:102B70006D3C0000DD2A0000692A000010B5044603
:102B8000003818BF01200549054B5322984704F12E
:102B90000800044B9847002010BD00BFC74F00003D
:102BA00039290000993C000038B50D46044610B1A3
:102BB000081E18BF01200349034B692298472C6067
:102BC000002038BDC74F000039290000014B012209
:102BD0005A717047000800400B4A937882B0DBB20C
:102BE0000193019B990705D5084B1B6813B15068E9
:102BF00002B01847019BDB0704D5044B5B680BB19F
:102C0000014AF4E702B0704700000241300500209D
:102C1000F8B5C46A05460E46174604B9F8BD6368A0
:102C20003A463146284698472468F6E738B590F882
:102C30003E309B07054601D1446B04B938BD63683B
:102C40002146284698472468F7E7000013B5846BAF
:102C50008023237006236370092A4FF00003237139
:102C60006371134638BF0923E38041F400714FF4C8
:102C7000FA736180009321461346006A04F10C0246
:102C8000014CA04702B010BDA126000013B5846B13
:102C900009220023627032222370618023716371E4
:102CA000A371E371009221461A46024C006AA047C4
:102CB00002B010BDA126000013B5846B80232370E1
:102CC000062363700023A3702371637101224FF404
:102CD000FA73E270E180009304F10C020B46006A83
:102CE0002146024CA04702B010BD00BFA126000043
:102CF000F8B54C68094F06460D4604B9F8BD63683F
:102D00001BB100220221204698472368A660214675
:102D10006B6006F11800B8476C68EEE7E528000024
:102D200013B58B79CC79006A03EB04239BB24AB1CB
:102D3000002B14BF4FF4FA7432240094024CA047C5
:102D400002B010BD3224F8E7A126000028B190F8A7
:102D50003E3023F0070380F83E30704770B5124BC9
:102D60009847062906460D46144619D80F4B1146BA
:102D70009847022D04BF04232374237C03F00F0320
:102D8000042B03D9237C43F0100323743046084BF3
:102D90002246294698473046064BBDE87040184702
:102DA0000729F3D10423F0E74D2D0000F12C00009A
:102DB000112C00002D2C0000F0B5846994F83E30F1
:102DC0000D46012161F3010385B0064684F83E30CB
:102DD000042A00F2B880DFE802F003B694A92900C3
:102DE0005A4B002229469847064660B194F83E3077
:102DF000606943F0040384F83E30554B294605B022
:102E0000BDE8F0401847A37BAB42524B40F09680A0
:102E1000214620469847627AA38C26749B1AA38485
:102E2000A673224601214C4B104664E0474F09220D
:102E30002946B84730BB0A2229463046B847002801
:102E400014BF02220122A37BAB421DD1E37B9B076F
:102E500003D1A38C627A9B1AA384226A0ABB012342
:102E60000393E37B0092C3F38103CDE90123114671
:102E700060693A4D4023A8470246206270B9092193
:102E8000204637E00022DEE74023237309236381D5
:102E9000E37BA57362F38303E373DEE73049314BD1
:102EA0009847E27B304E00250323C2F3810223744E
:102EB0006572237B00922946206A2A46B047014664
:102EC000E8B9E37B13F00C0F09D0322384F83F30CC
:102ED000264A6069264B05B0BDE8F0401847217BC3
:102EE000244B122928BF12212046984758B3224666
:102EF00005212046204B05B0BDE8F04018472A4682
:102F0000BDE7124B022229469847A37BAB421AD158
:102F1000114D237C38B143F020032374224606214F
:102F200020462B46E7E760F34513F6E7A37BAB4269
:102F300009D1042323742246022174E70146204666
:102F40009847737AFFDE05B0F0BD00BF3F22000056
:102F500031220000F12C0000112C00009922000009
:102F6000ED2F00007D260000512500007D2F000080
:102F7000291A0000B92C00005D2D000038B58469C5
:102F800094F83F10D9B10139C9B284F83F10B1B9F2
:102F9000237C042B16D8217B104B122928BF122129
:102FA00020469847A26A05461AB960690C4B11463B
:102FB000984725B10B4B2246052120469847A56A24
:102FC0002DB938BD6289084B20469847EAE76B68FF
:102FD0002946204698472D68F2E700BFB92C00002B
:102FE000291A00005D2D00004D2C00002DE9F04F46
:102FF000C67B85B0002E78D103689C6994F83E307A
:1030000003F00303012B40F0F48090F92730002BEC
:1030100007DA2246072110467C4B05B0BDE8F04F89
:103020001847A56B6F78062F1BD0092F00F0C780BB
:10303000052F5AD1E27B237B617B2774C2F3810287
:103040000092206A724D3246A847002814DB714A6C
:103050006069714B84F83F70314605B0BDE8F04FB0
:1030600018476988090A012942D1206A90F9273056
:1030700013B9C28B072A02D822460521CBE7EF7C81
:103080002773112A14D8E67BC27B817BC6F38106A5
:1030900000963B465E4EB04718B9604B1221204661
:1030A0009847002821DA05F10C0209212046B3E7F0
:1030B0002A7D2A72A26B697D5172A26BA97D9172E1
:1030C000A26BE97DD172A16B627B4A800525322219
:1030D0000B704D700B714B718B71CB710092206A2C
:1030E0004F4E1A46B0470028C6DB05B0BDE8F08F4A
:1030F0000229FAD1236ADB8B082BBDD9092B0ED10B
:10310000EB8963819AB2A38F083B9A4202D9224687
:10311000042180E7434B314620469847E3E72A7D68
:10312000A38C62721344FA2B20DD384B22462046D2
:103130009847A36B3C4FDA7B997BDFF8F890DFF878
:10314000FCA0DFF8FCB003F10C0001EB022110FA47
:1031500081F104220391B847B8460290029B3BB923
:1031600056B3697C314B20469847BCE7A384E0E71F
:10317000A76947B902AA0A212046C847029B1A78C4
:103180001344029310E07B68A3B102AA00213846E1
:10319000984778B93946BC6004F11800D0473946E1
:1031A000201DD8470136F6B2DDE902010422C047EE
:1031B0000290D3E73F68DCE7224603212BE7162382
:1031C000237420461A4B9847656855B9194B224617
:1031D000294620469847184B204605B0BDE8F04FD9
:1031E00018476B681BB100220121284698472D68BB
:1031F000EBE70F4B20469847256B002DEBD06B6813
:1032000013B1216A204698472D68F6E75D2D00002E
:10321000512500007D2F0000291A0000B92C000064
:10322000A12600004D2C0000D13400008D2C0000A0
:103230004D2D0000112C00002D2C00001129000044
:10324000E5280000022AF7B504460D4608D1037CA4
:10325000D90629D5037C9B0603D56FF004001DE039
:1032600028B394F83E3013F0030623D162F3010330
:1032700084F83E30E37B617B206A114FC3F3810306
:1032800000933246237BB847002809DA94F83E3091
:1032900066F3010384F83E306FF0050003B0F0BD23
:1032A0005DB12C603046F9E76FF01000F6E76FF083
:1032B0001300F3E76FF00300F0E72846EEE700BFE6
:1032C000512500002DE9F0410E4617469846044668
:1032D00038B100292ED0002A2ED0202B94BF0020F8
:1032E00001201849184B40F234529847A56B2DBB6A
:1032F000402323736661B461E289144B256022F494
:103300009F52012122F01F02E281C4E90A55C4E95B
:103310000C550F4AA561A5846560617365813046CF
:103320009847A763A4F83C8084F83E50257428464B
:10333000BDE8F0810846D4E71046D2E76FF01100EF
:10334000F6E700BFE34F000039290000291A00000A
:10335000B92D000070B50D46044610B1081E18BF07
:1033600001200A4B0A4940F2A5529847237C03F0FA
:10337000FF063BB904F11800064B29469847AC609C
:10338000304670BD6FF01000FBE700BF3929000028
:10339000E34F0000E528000070B50D4616460446D0
:1033A00020B172B15068003818BF01201649174B80
:1033B00040F2BD529847032D25D8DFE805F00417E9
:1033C00020221046F2E704F12805114B3146284629
:1033D0009847C0B9A16A19B90E4A60690E4B98475F
:1033E00031462846BDE870400C4B18472C34084B3A
:1033F00031462046984730B931462046F2E730340E
:10340000F5E73434F3E770BDE34F000039290000DD
:10341000D52800007D2F0000291A0000E5280000B3
:1034200070B50E461546044610B1101E18BF012097
:103430001349144B40F2E1529847032E1FD8DFE89E
:1034400006F0020F161A104B294604F1280098477F
:10345000A26AA2B960690D4BBDE8704011461847D9
:10346000294604F12C00BDE87040074B1847294657
:1034700004F13000F7E7294604F13400F3E770BDAA
:10348000E34F00003929000011290000291A00002B
:1034900010B50446003818BF01200349034B40F221
:1034A0001B729847204610BDE34F000039290000E9
:1034B00010B50446003818BF01200349034B40F201
:1034C00021729847A06810BDE34F00003929000021
:1034D00010B5884201D3002010BD0378012BFAD922
:1034E00044789442F8D01844F3E710B5884201D3E9
:1034F000084610BD0378012B07D94478042C02D16B
:1035000084789442F5D11844F0E70020F1E788422E
:1035100001D3002070470378012BFAD94278042A9E
:10352000F7D0052AF6D01844F1E7704708B50E4BDE
:1035300098470E4B98470E4B0E48D3F8802042F028
:103540008052C3F88020D3F8902042F08052C3F814
:103550009020D3F8902022F08052C3F89020064BA0
:103560009847064B9847FEE7DD3F000065400000A6
:10357000008000416C050020ED150000BD07000033
:10358000064B42F28E029A8200229A75DA75DA6947
:1035900002F47C52DA6101221A7470470014004070
:1035A00003690B42FCD1704710B5044618B100689E
:1035B000003818BF01201749174B2F229847174B87
:1035C0002068174A1C6048F20301904703889B0754
:1035D0000AD52068038823F002031B041B0C038018
:1035E0009047206802219047206803889BB243F0EF
:1035F00001030380012190472068904720684FF421
:103600000143038048F203019047236800201866B5
:1036100010BD00BFF74F0000392900004005002011
:10362000A13500000D4B10B51C68226891895389A3
:103630009BB20B40DA0507D563682046984723689C
:103640004FF480729A8110BD5B04FCD5A3682046BC
:10365000984723684FF48042F4E700BF40050020FC
:1036600000F01F0330B501259D4040090D4BC001FE
:103670000229ACB24FEA154203440BD044F0804417
:1036800044F4003442F040425D6042F400329C62F7
:103690009A6230BD44F080449D6042F040429C629A
:1036A000F6E700BF00800041420900F01F0303EB72
:1036B000C21303F1824303F5004393F8402002F064
:1036C000FB0283F8402070474309DB0103F182438A
:1036D00030B503F5004300F01F041D1903EB54033C
:1036E00095F8402002F0FE0242F0010285F84020E9
:1036F000CAB293F8301010F0010F1BBF01F00F0198
:1037000041EA021101F0F001C9B208BF114383F888
:10371000301030BD2DE9F04101211E4E1E4D1F4CD1
:103720001F4F2B20B0472B201E49A847A04702213E
:103730000820B0474FF480737B6108201A49A847DE
:10374000A04702210920B0474FF400737B61092094
:103750001649A847A04702210A20B0474FF48063CA
:103760007B610A201249A847A04702210B20B047DD
:103770004FF400637B610B200E49A847A04701214D
:103780002A20B0472A20A8470B492346BDE8F0412C
:10379000184700BF61360000A9360000C936000096
:1037A0000080004107002B00070008000700090007
:1037B00007000A0007000B0007002A00064B1A69E1
:1037C00042F400521A611A6942F400121A61DA696D
:1037D00042F40052DA6170470008004010B5054B12
:1037E000054906489847064B9847BDE81040054BE9
:1037F000184700BFBD3700000034004248050020D4
:10380000193F000015370000024A536943F4007362
:10381000536170470008004010B5044B0449054847
:103820009847BDE81040044B184700BF0938000016
:10383000002400404C0500200903000070B5124E22
:10384000124D134C4FF08063C6F8943002213A2099
:10385000A84701F568113A20A0474FF00063C6F869
:10386000943002213B20A84701F56C113B20A04772
:1038700001213D20A847074B07493D209847234693
:10388000BDE87040184700BF00800041613600006D
:10389000C9360000A936000002003D00064B402258
:1038A000C3F8DC204322C3F88C20044A936943F414
:1038B00000739361704700BF001C00400008004087
:1038C00010B5054B054906489847064B9847BDE893
:1038D0001040054B184700BF9D38000000200141F3
:1038E0006C050020A11500003D38000010B5054C06
:1038F00005492C20A04723460449BDE810402D204F
:10390000184700BFC936000002002C0002002D003D
:10391000064B4022C3F808214322C3F88C20044AF6
:10392000136A43F001031362704700BF001C00409C
:103930000008004010B5064B064898474FF08641F6
:10394000054B00229847BDE81040044B184700BFC4
:1039500011390000840500203D2B0000ED380000E7
:103960002DE9F047224E234F234D244C4FF40018ED
:1039700002211520B84715202149C6F81480A84710
:103980004FF48019A04702211420B84714201D4984
:10399000C6F81490A847A04702213220B8474FF438
:1039A0008023C6F8943032201749A847A047022147
:1039B0003320B8474FF40023C6F89430332013491E
:1039C000A847A04702213420B84734201049C6F840
:1039D0009490A847A04702213520B847C6F89480A4
:1039E0003520A8470B492346BDE8F047184700BFDC
:1039F0000080004161360000A9360000C936000091
:103A00000800150008001400080032000800330008
:103A10000800340008003500054A136943F4803378
:103A20001361044B4022C3F83821C3F88C2070473F
:103A300000080040001C004010B5054B05489847A1
:103A40004FF08C41044B9847BDE81040034B18479A
:103A5000193A0000900500200D17000061390000A0
:103A600070470000074B4022C3F8A820A3F5A053DD
:103A70001A6942F480621A619A6942F001029A61FD
:103A8000704700BF001C00402DE9F04102210D4F9E
:103A90000D4E0E4D0E4C1820B8474FF080737361D9
:103AA00018200C49A847A04702211920B8474FF019
:103AB000007373611920A84707492346BDE8F04108
:103AC000184700BF6136000000800041A9360000A1
:103AD000C9360000070018000700190010B5064B92
:103AE000064898474FF08241054B00229847BDE8B1
:103AF0001040044B184700BF653A0000A80500209D
:103B0000C5180000893A000010B5084B9847084BCB
:103B10009847084B9847084B9847084B9847084BDD
:103B20009847BDE81040074B184700BF55280000D4
:103B3000DD37000019380000C138000035390000B9
:103B4000393A0000DD3A0000C3690B42FCD17047EE
:103B5000C3690B42FCD170470268034B22F002029A
:103B600002600321184700BF493B00000268034B75
:103B700022F0020202600321184700BF513B0000FF
:103B800070B50C4D06460FCD88B06C460FC495E855
:103B90000F0084E80F006A46002352F8041BB1426C
:103BA00002D1D8B208B070BD0133082BF5D1002086
:103BB000F8E700BF28500000C26912F0010208B502
:103BC00008D1036843F0020303600321034B9847C5
:103BD000104608BD6FF00300FBE700BF493B000043
:103BE00038B51B4B04469847042805D019491A4B91
:103BF00040F2472200209847E369184D13F0010F67
:103C00000ED103212046A84723689B0703D5144BF8
:103C100098470221A8470523236003212046A8478F
:103C200020460121A8470F4B23600321A8474FF4EA
:103C3000403363601F21A8470B4BA3604FF22963F9
:103C4000A3810023A373184684F8303038BD00BF29
:103C5000813B00000C50000039290000513B00005E
:103C60006D3B0000040010400200700070B5054676
:103C700000380C46054B064918BF0120BB22984767
:103C80002C602046034BBDE87040184739290000DE
:103C90000C500000E13B00000068036843F00203A1
:103CA00003600321004B1847513B000003689962F1
:103CB00070470368986AC0B270470368187E00F0C6
:103CC000010070470368187EC0F340007047036826
:103CD000187EC0F3800070472DE9F843444B454DF2
:103CE000074608460C469847022818BF0025002FB3
:103CF0005DD0201E18BF01203F4E404940F63F12C4
:103D0000B047B046002D70D0E3693D4E13F0010F6F
:103D100013D103212046D5F80090B04723689B07B4
:103D200009F01C0903D5374B98470221B04749F0E9
:103D30000103236003212046B04701212046B047FC
:103D40002B68DFF8C4903C6003F01C03082B30D1D3
:103D50002A49012040F61D12C0472B6803EA0903D7
:103D6000236003212046B0476B6823F4083323F413
:103D7000107343F4003343F4107363601721B047AA
:103D8000AB6863626B7B84F83030E369002BFCD155
:103D90006B6813F0070F0CBF012302233B71AB7B51
:103DA000EA7B43EA0223FB800020BDE8F883384623
:103DB000A2E71249012040F60912C0472B6803EA26
:103DC0000903236003212046B0476B6823F438338E
:103DD00023F4107343F4003363601721B0472B7B47
:103DE00023736B7B84F83030D2E76FF00C00DCE794
:103DF000813B000060500000392900000C50000099
:103E0000493B0000593B0000FCFEFFFF10B5044693
:103E100018B10068003818BF0120054B054940F66D
:103E20009E1298472068044BBDE81040184700BF19
:103E3000392900000C500000B93B00002DE9F8437F
:103E4000046890F804802A4B0746201ED1E90065DB
:103E500040F6A32218BF0120894626499847E26907
:103E600012F007023ED1244B0321204698472368D5
:103E700099073AD51146237ED8B25B070FD48A4200
:103E800018D8C30716D5FB8836B1B8F1010F3378BF
:103E90008CBF36F8023B01360132A3620AE0A36A06
:103EA0003DB1B8F1010F2B7085BF1B0A6B70013556
:103EB00002350131000607D4D9F808309342DAD828
:103EC0008B42D8D8104606E04FF6FF7363838023F9
:103ED00023766FF01200237E9B07FCD0032323760A
:103EE000BDE8F8836FF00300FAE76FF01300F7E71F
:103EF000392900000C500000493B0000EFF310830B
:103F0000036072B6BFF35F8F7047BFF35F8F0368C4
:103F100083F310887047000070B50D46044610B159
:103F2000081E18BF01200549054B31229847294634
:103F30002046044BBDE87040184700BF7150000098
:103F400039290000D5020000FEE700001849194891
:103F5000814210B50AD0184BDA1C121A22F0030263
:103F6000C41EA34238BF0022144B9847144B154877
:103F7000DA1C121AC11E22F00302994288BF0022E5
:103F8000114B00219847114A114B22F07F029A6091
:103F9000D3F8882042F47002C3F88820BFF34F8F13
:103FA000BFF36F8F0B4B98470B4B9847FEE700BF53
:103FB000785100000000002074000020FD40000047
:103FC000E0050020780000201941000000000000FA
:103FD00000ED00E0B54000002D35000010B5054BA8
:103FE0009847054B9847054B9847BDE81040044B50
:103FF000184700BF093B0000210800002B350000D6
:10400000D91600000FB430B5C3B0114C469D2846F8
:10401000A047FF2818D80F4B4FF48072002102A848
:10402000984747AA0C4B0192294602A8984702A834
:10403000A0470A4B82B202A91868094B984743B0BF
:10404000BDE8304004B070474FF0FF30F7E700BFE5
:10405000294100001941000065410000C40500200D
:10406000A502000010B5064C0649074B20469847AC
:10407000064B20469847064B06489847002010BD3F
:1040800084050020C4050020A92B00007D2B000022
:10409000054000008C50000010B50C46194620B9B0
:1040A00023460248024CA047FEE710BD9F50000087
:1040B0000540000070B50D4D0D4C641BA41000268A
:1040C000A64209D10B4D0C4C01F046F8641BA4101C
:1040D0000026A64205D170BD55F8043B984701362D
:1040E000EEE755F8043B98470136F2E764510000CB
:1040F0006451000064510000685100000A4491427C
:1041000000F1FF3300D1704710B511F8014B03F8EF
:10411000014F9142F9D110BD02440346934200D1B0
:10412000704703F8011BF9E7034613F8012B002A37
:10413000FBD1181A0138704700B59BB0009104916B
:104140006FF000410591029105490391694600F025
:10415000CBF8009B00221A701BB05DF804FB00BF77
:104160000802FFFF13460A46014602480068FFF7AF
:10417000E3BF00BF1000002070477047F8B5CD1CAA
:1041800025F0030508350C2D38BF0C25002D0646FB
:1041900001DBA94203D90C2333600020F8BD00F0F5
:1041A000B1FB21490A6814469CB9204F3B6823B9EA
:1041B0002146304600F02CFB38602946304600F09E
:1041C00027FB431C23D10C233360304600F0A0FBB7
:1041D000E3E723685B1B17D40B2B03D923601C4434
:1041E000256004E06368A2420CBF0B605360304658
:1041F00000F08EFB04F10B00231D20F00700C21A13
:10420000CCD01B1AA350C9E722466468CCE7C41C73
:1042100024F00304A042E3D0211A304600F0F8FA5B
:104220000130DDD1CFE700BFC8050020CC0500205C
:104230002DE9F0478E689E4282460C4690461F4606
:1042400038D88A8912F4906F32D025680969A5EBB5
:104250000109656905EB450505EBD57501334B444F
:104260006D109D4238BF1D46530531D52946FFF7D5
:1042700085FF064650B90C23CAF80030A38943F0E5
:104280004003A3814FF0FF30BDE8F08721694A4623
:10429000FFF734FFA38923F4906343F08003A381E5
:1042A000266165614E44A5EB09052660A5603E4682
:1042B000BE4200D93E4632462068414600F008FB27
:1042C000A36822689B1B3244A36022600020DBE7C6
:1042D0002A4600F071FB06460028E1D121695046CC
:1042E00000F01CFBC7E700002DE9F04F98468B89D2
:1042F0001B069DB007460D4614460ED50B6963B9E3
:104300004021FFF73BFF2860286120B90C233B6068
:104310004FF0FF30D1E040236B610023099320234D
:104320008DF82930CDF80C803023DFF8A8818DF886
:104330002A304FF0010923469A4613F8012B0AB19F
:10434000252AF9D1BAEB040B0BD05B46224629464D
:104350003846FFF76DFF013000F0AA80099A5A44F1
:1043600009929AF80030002B00F0A28000234FF051
:10437000FF32CDE905230AF1010A049307938DF872
:1043800053301A935446052214F8011B514800F08B
:104390004FFA049AD8B9D00644BF20238DF8533081
:1043A000110744BF2B238DF853309AF800302A2B85
:1043B00015D0079A544600204FF00A0C214611F8F8
:1043C000013B303B092B4ED9B0B1079214E0A0EB72
:1043D000080309FA03F313430493A246D2E7039BAD
:1043E000191D1B680391002BBBBF5B4242F0020208
:1043F00007930793B8BF049223782E2B0CD16378D0
:104400002A2B35D1039B1A1D1B680392002BB8BFC2
:104410004FF0FF3302340593DFF8C8A02178032260
:10442000504600F005FA40B14023A0EB0A0003FA21
:1044300000F0049B03430134049314F8011B264845
:104440008DF82810062200F0F3F9002838D0234B0D
:104450001BBB039B073323F0070308330393099B1C
:104460003344099367E70CFB02320C460120A5E7B1
:1044700000230134059319464FF00A0C204610F82A
:10448000012B303A092A03D9002BC5D00591C3E787
:104490000CFB012104460123F0E703AB00932A46FD
:1044A0000F4B04A93846AFF30080421C0646D6D114
:1044B000AB895B063FF52CAF09981DB0BDE8F08FC6
:1044C00003AB00932A46064B04A9384600F07AF85D
:1044D000EBE700BF245100002E5100000000000057
:1044E000314200002A5100002DE9F0471646994656
:1044F0008A680B69DDF820809342B8BF13463360A9
:1045000091F8432007460C460AB101333360236813
:10451000990642BF336802333360256815F00605FB
:1045200006D104F1190AE36832689B1AAB4226DC13
:1045300094F84320131E226818BF012392062BD43F
:1045400004F1430249463846C04701301ED0236873
:10455000E568326803F00603042B08BFAD1AA368B0
:1045600022690CBF25EAE57500259342C4BF9B1A5A
:10457000ED1800261A34B5421AD1002008E00123B4
:10458000524649463846C047013003D14FF0FF300C
:10459000BDE8F0870135C6E7E1185A1C302081F8E4
:1045A0004300224494F8451082F843100233C7E7D1
:1045B0000123224649463846C0470130E6D001363D
:1045C000D9E700002DE9FF470C469146277E0C995C
:1045D000782F80469A4604F1430207D8622F0AD802
:1045E000002F00F0D880582F00F0A38004F142067D
:1045F00084F842703AE0A7F16303152BF6D801A0C6
:1046000050F823F05D46000071460000ED450000C3
:10461000ED450000ED450000ED450000714600004D
:10462000ED450000ED450000ED450000ED450000C2
:104630007D470000A14600005F470000ED450000F7
:10464000ED4500009F470000ED450000A146000039
:10465000ED450000ED450000674700000B681A1D9E
:104660001B680A6004F1420684F842300123A3E08B
:10467000256808682E0600F104030AD505680B605A
:10468000002D03DA2D236D4284F843305E480A235F
:1046900019E015F0400F05680B6018BF2DB2EFE769
:1046A0000B682568181D0860280601D51D6802E002
:1046B0006906FBD51D8854486F2F0CBF08230A23B9
:1046C000002184F843106668A660002EA2BF21680E
:1046D00021F0040121600DB9002E4DD01646B5FB26
:1046E000F3F103FB1157C75D06F8017D2F46BB426E
:1046F0000D46F4D9082B0BD12368DF0708D52369B1
:1047000061689942DEBF302306F8013C06F1FF36AE
:10471000921B2261CDF800A04B4603AA21464046D9
:10472000FFF7E2FE01304CD14FF0FF3004B0BDE89E
:10473000F087354884F8457023680E681F0656F8E0
:10474000045B0E6014D5D90744BF43F020032360F7
:104750001DB9236823F0200323601023B0E72368EA
:1047600043F0200323607823284884F84530E3E7AA
:104770005E0648BFADB2E6E71646BBE70B682668A3
:1047800060691D1D0D6035061B6801D5186002E0CB
:104790007106FBD51880002323611646BAE70B6823
:1047A0001A1D0A601E6862680021304600F040F859
:1047B00008B1801B606063682361002384F8433084
:1047C000A8E72369324649464046D0470130ABD07E
:1047D00023689B0713D4E068039B9842B8BF184630
:1047E000A4E70123324649464046D04701309BD0DA
:1047F0000135E36803995B1AAB42F2DCEBE7002575
:1048000004F11906F5E700BF3551000046510000DC
:1048100038B5064D0023044608462B60FCF70CF81B
:10482000431C02D12B6803B1236038BDDC05002096
:1048300001F0FF01102A2BDB10F0070F08D010F851
:10484000013B013A8B422DD010F0070F42B3F6D155
:10485000F0B441EA012141EA014122F007047FF06E
:1048600000070023F0E80256083C85EA010586EAC5
:10487000010685FA47F5A3FA87F586FA47F6A5FA01
:1048800087F68EB9EED1F0BC01F0FF0102F007020D
:1048900032B110F8013B013A83EA010313B1F8D1B8
:1048A0000020704701387047002D06BF3546033899
:1048B000073815F0010F07D1013015F4807F02BFD2
:1048C000013015F4C03F0130F0BC0138704700BF23
:1048D000884210B501EB020402D98442234607D86E
:1048E000431EA14208D011F8012B03F8012FF8E76D
:1048F000024401468A4200D110BD13F8014D02F86E
:10490000014DF7E70148FFF737BC00BFD405002091
:104910000148FFF732BC00BFD405002038B505467A
:10492000002945D051F8043C0C1F002BB8BFE418F7
:10493000FFF7E8FF1F4A1368104633B9636014603D
:104940002846BDE83840FFF7E3BFA3420BD92168F2
:104950006218934204BF1A685B68636004BF521810
:1049600022600460ECE71A465B680BB1A342FAD9F7
:1049700011685018A0420BD120680144501883429E
:104980001160DDD118685B68536001441160D7E79E
:1049900002D90C232B60D3E7206821188B4204BF77
:1049A00019685B68636004BF091821605460C7E739
:1049B00038BD00BFC8050020F8B5074614460E46AE
:1049C00021B9BDE8F8401146FFF7D8BB22B9FFF77F
:1049D000A5FF25462846F8BD00F014F8A0420FD2E6
:1049E00021463846FFF7CAFB05460028F2D031467B
:1049F0002246FFF783FB31463846FFF78FFFE9E792
:104A00003546E7E751F8043C181F002BBCBF0B5894
:104A1000C01870472E2E2F68616C2F7372632F6839
:104A2000616C5F696F2E63002E2E2F68706C2F7182
:104A30007370692F68706C5F717370692E63002EDC
:104A40002E2F68616C2F7372632F68616C5F6361D6
:104A50006C656E6461722E63004552523A20256483
:104A60000A002E2E2F73645F6D6D632F73645F6D6C
:104A70006D632E63003E3E3E00537461727420539A
:104A800044206361726420696E7374616C6C0A0DFA
:104A90000025733A20434D443535204661696C0A40
:104AA0000D0025733A2041434D443431204661695D
:104AB0006C0A0D0025733A2041434D443431205493
:104AC000696D656F7574206F6E20627573792C2027
:104AD00072657370333220307825303878200A0DB3
:104AE0000025733A20434D443538204661696C0AED
:104AF0000D005374617274204D4D4320496E7374E0
:104B0000616C6C0A0D0025733A20434D44312053EB
:104B10005049204661696C202D20427573792072BE
:104B2000657472792025640A0D0025733A20434D7F
:104B300044312054696D656F7574206F6E20627505
:104B400073790A0D0053442F4D4D43206361726405
:104B50002072656164790A0D0000000073645F7360
:104B600070695F6F705F636F6E64006D6D635F731C
:104B700070695F6F705F636F6E640000000000001B
:104B80000A0000000C0000000D0000000F000000F3
:104B9000140000001A0000001E00000023000000A6
:104BA000280000002D000000340000003700000045
:104BB0003C00000046000000500000000A00000019
:104BC00064000000E803000010270000000000005F
:104BD0000000000000000000000000000A000000CB
:104BE0000C0000000D0000000F0000001400000089
:104BF000190000001E000000230000002800000033
:104C00002D00000032000000370000003C000000D2
:104C100046000000500000002E2E2F73645F6D6D63
:104C2000632F73645F6D6D635F7370692E6300251E
:104C3000733A205265616420626C6F636B732074F9
:104C4000696D656F75740A0D0025733A20435243F0
:104C50002064617461206572726F7220746F6B657D
:104C60006E0A0D0025733A204F7574206F6620720E
:104C7000616E67652064617461206572726F722075
:104C8000746F6B656E0A0D0025733A20496E76616C
:104C90006C6964204461746120526573706F6E7337
:104CA0006520546F6B656E20307825780A0D0025DD
:104CB000733A20577269746520626C6F636B732C52
:104CC0002053445F4D4D435F5350495F4552525FFF
:104CD0004352432C207265737020307825780A0D7A
:104CE0000025733A20577269746520626C6F636B9C
:104CF000732053445F4D4D435F5350495F455252BB
:104D00005F57522C207265737020307825780A0D19
:104D10000025733A2053746F702077726974652090
:104D2000626C6F636B732074696D656F75740A0DC7
:104D3000004E6F205344204361726420726573708B
:104D40006F6E7365207761732070726573656E7422
:104D50002E2E2E0025733A20636D64202530326498
:104D60002C206172672030782530386C582C205206
:104D7000312074696D656F75740D0A0025733A20D2
:104D8000636D6420253032642C2061726720307896
:104D90002530386C782C20723120307825303278EC
:104DA0002C2052315F5350495F434F4D5F43524374
:104DB0000A0D0025733A20636D6420253032642C7F
:104DC000206172672030782530386C782C20723161
:104DD00020307825782C20523120494C4C454741D1
:104DE0004C5F434F4D4D414E440A0D0025733A2010
:104DF000636D6420253032642C2061726720307826
:104E00002530386C782C20723120307825782C2091
:104E10005231206572726F720A0D0025733A206359
:104E20006D6420253032642C206172672030782533
:104E300030386C782C2042757379207369676E6105
:104E40006C20616C7761797320686967680A0D006E
:104E500025733A20577269746520626C6F636B73B7
:104E60002074696D656F75740A0D003C3C3C0073DD
:104E700070695F6D5F73796E635F73746172745F85
:104E8000726561645F626C6F636B007370695F6D04
:104E90005F73796E635F73746F705F777269746547
:104EA0005F626C6F636B007370695F6D5F73796EC7
:104EB000635F73746F705F6D756C7469777269741A
:104EC000655F626C6F636B007370695F6D5F7379B0
:104ED0006E635F616474635F737461727400737096
:104EE000695F6D5F73796E635F73746172745F770E
:104EF000726974655F626C6F636B73007370695F76
:104F00006D5F73796E635F776169745F656E645F0F
:104F10006F665F77726974655F626C6F636B730055
:104F20007370695F6D5F73796E635F7772697465C3
:104F30005F776F7264002E2E2F68616C2F7372631F
:104F40002F68616C5F7370695F6D5F73796E632E3C
:104F500063002E2E2F68616C2F7372632F68616C53
:104F60005F6D63695F73796E632E63002E2E2F6809
:104F7000706C2F7573622F68706C5F7573622E632F
:104F80000000080010002000400080000001000226
:104F900000042E2E2F68616C2F7574696C732F734B
:104FA00072632F7574696C735F6C6973742E630020
:104FB0002E2E2F68706C2F736468632F68706C5F7F
:104FC000736468632E63002E2E2F68616C2F7372DA
:104FD000632F68616C5F75736172745F73796E6360
:104FE0002E63002E2E2F7573622F686F73742F75CA
:104FF000736268632E63002E2E2F68706C2F72749C
:10500000632F68706C5F7274632E63002E2E2F689E
:10501000706C2F736572636F6D2F68706C5F736552
:1050200072636F6D2E63000000300040003400405A
:105030000020014100400141000000430004004302
:1050400000080043000C00430000000000000000C6
:105050000000000000000000000000000000000050
:105060000C0030000000020000000000FE00FF0005
:10507000022E2E2F68616C2F7372632F68616C5F34
:10508000717370695F73796E632E63004465627536
:105090006720496E697469616C697A65640A0041C8
:1050A0007373657274204661696C757265206174F2
:1050B000206C696E652025642C2025733A202573A9
:1050C0000A000000000000000000000000000000D6
:1050D00000000000000000000000000000000000D0
:1050E00000000000000000000000000000000000C0
:1050F00000000000000000000000000000000000B0
:10510000000000000000000000000000000000009F
:10511000000000000000000000000000000000008F
:1051200000000000232D302B2000686C4C006566C9
:1051300067454647003031323334353637383941E8
:1051400042434445460030313233343536373839FE
:105150006162636465660000F8B500BFF8BC08BC16
:105160009E46704789020000F8B500BFF8BC08BC35
:085170009E4670476502000035
:105178000000000081040000FFFF0100FFFF0100A4
:105188001400002000000000E4500000045100005A
:10519800C4500000000000000000000000000000F3
:1051A80000000000000000000000000000000000F7
:1051B80000000000000000000000000000000000E7
:1051C80000000000000000000000000000000000D7
:1051D80000000000000000000000000000000000C7
:0451E80000000000C3
:00000001FF
